BL51 BANKED LINKER/LOCATER V5.03                                                        06/13/2014  14:13:10  PAGE 1


BL51 BANKED LINKER/LOCATER V5.03, INVOKED BY:
D:\KEIL\C51\BIN\BL51.EXE liu.obj, .\USBJmpTb.OBJ TO liu RAMSIZE (256)


MEMORY MODEL: SMALL


INPUT MODULES INCLUDED:
  liu.obj (LIU)
  .\USBJmpTb.OBJ (USBJMPTBL)
  D:\KEIL\C51\LIB\C51S.LIB (?C_STARTUP)


LINK MAP OF MODULE:  liu (LIU)


            TYPE    BASE      LENGTH    RELOCATION   SEGMENT NAME
            -----------------------------------------------------

            * * * * * * *   D A T A   M E M O R Y   * * * * * * *
            REG     0000H     0008H     ABSOLUTE     "REG BANK 0"
            IDATA   0008H     0001H     UNIT         ?STACK

            * * * * * * *   C O D E   M E M O R Y   * * * * * * *
            CODE    0000H     0003H     ABSOLUTE     
            CODE    0003H     001DH     UNIT         ?PR?DELAY?LIU
            CODE    0020H     000FH     UNIT         ?PR?MAIN?LIU
            CODE    002FH     000CH     UNIT         ?C_C51STARTUP
                    003BH     0008H                  *** GAP ***
            CODE    0043H     0003H     ABSOLUTE     
                    0046H     000DH                  *** GAP ***
            CODE    0053H     0003H     ABSOLUTE     
                    0056H     00AAH                  *** GAP ***
            CODE    0100H     00B8H     PAGE         ?PR?USB_JUMP_TABLE?USBJT



OVERLAY MAP OF MODULE:   liu (LIU)


SEGMENT
  +--> CALLED SEGMENT
---------------------
?C_C51STARTUP
  +--> ?PR?MAIN?LIU

?PR?MAIN?LIU
  +--> ?PR?DELAY?LIU



UNRESOLVED EXTERNAL SYMBOLS:
   ISR_EP0ACK
   ISR_EP0IN
   ISR_EP0OUT
   ISR_EP0PINGNAK
   ISR_EP1IN
   ISR_EP1OUT
BL51 BANKED LINKER/LOCATER V5.03                                                      06/13/2014  14:13:10  PAGE 2


   ISR_EP1PINGNAK
   ISR_EP2EFLAG
   ISR_EP2FFLAG
   ISR_EP2INOUT
   ISR_EP2PFLAG
   ISR_EP2PIDERROR
   ISR_EP2PINGNAK
   ISR_EP4EFLAG
   ISR_EP4FFLAG
   ISR_EP4INOUT
   ISR_EP4PFLAG
   ISR_EP4PIDERROR
   ISR_EP4PINGNAK
   ISR_EP6EFLAG
   ISR_EP6FFLAG
   ISR_EP6INOUT
   ISR_EP6PFLAG
   ISR_EP6PIDERROR
   ISR_EP6PINGNAK
   ISR_EP8EFLAG
   ISR_EP8FFLAG
   ISR_EP8INOUT
   ISR_EP8PFLAG
   ISR_EP8PIDERROR
   ISR_EP8PINGNAK
   ISR_ERRORLIMIT
   ISR_GPIFCOMPLETE
   ISR_GPIFWAVEFORM
   ISR_HIGHSPEED
   ISR_IBN
   ISR_SOF
   ISR_STUB
   ISR_SUDAV
   ISR_SUSP
   ISR_SUTOK
   ISR_URES



SYMBOL TABLE OF MODULE:  liu (LIU)

  VALUE           TYPE          NAME
  ----------------------------------

  -------         MODULE        LIU
  C:0000H         SYMBOL        _ICE_DUMMY_
  C:0003H         PUBLIC        delay
  C:0020H         PUBLIC        main
  D:00B2H         PUBLIC        OEA
  D:0080H         PUBLIC        IOA
  -------         PROC          MAIN
  C:0020H         LINE#         7
  C:0020H         LINE#         8
  C:0020H         LINE#         9
  C:0023H         LINE#         10
  C:0026H         LINE#         11
  C:0029H         LINE#         12
BL51 BANKED LINKER/LOCATER V5.03                                                      06/13/2014  14:13:10  PAGE 3


  C:002CH         LINE#         13
  -------         ENDPROC       MAIN
  -------         PROC          DELAY
  -------         DO            
  D:0006H         SYMBOL        i
  D:0004H         SYMBOL        k
  -------         ENDDO         
  C:0003H         LINE#         16
  C:0003H         LINE#         17
  C:0003H         LINE#         18
  C:0006H         LINE#         19
  C:0006H         LINE#         20
  C:0006H         LINE#         21
  C:0014H         LINE#         22
  C:001FH         LINE#         24
  -------         ENDPROC       DELAY
  -------         ENDMOD        LIU

  -------         MODULE        USBJMPTBL
  C:0100H         SEGMENT       ?PR?USB_JUMP_TABLE?USBJT
  N:0045H         PUBLIC        USB_INT2AUTOVECTOR
  N:0055H         PUBLIC        USB_INT4AUTOVECTOR
  C:0100H         PUBLIC        USB_JUMP_TABLE
  N:0000H         SYMBOL        USBJMPTBL
  C:0043H         LINE#         49
  C:0053H         LINE#         53
  C:0100H         LINE#         61
  C:0104H         LINE#         63
  C:0108H         LINE#         65
  C:010CH         LINE#         67
  C:0110H         LINE#         69
  C:0114H         LINE#         71
  C:0118H         LINE#         73
  C:011CH         LINE#         75
  C:0120H         LINE#         77
  C:0124H         LINE#         79
  C:0128H         LINE#         81
  C:012CH         LINE#         83
  C:0130H         LINE#         85
  C:0134H         LINE#         87
  C:0138H         LINE#         89
  C:013CH         LINE#         91
  C:0140H         LINE#         93
  C:0144H         LINE#         95
  C:0148H         LINE#         97
  C:014CH         LINE#         99
  C:0150H         LINE#         101
  C:0154H         LINE#         103
  C:0158H         LINE#         105
  C:015CH         LINE#         107
  C:0160H         LINE#         109
  C:0164H         LINE#         111
  C:0168H         LINE#         113
  C:016CH         LINE#         115
  C:0170H         LINE#         117
  C:0174H         LINE#         119
  C:0178H         LINE#         121
BL51 BANKED LINKER/LOCATER V5.03                                                      06/13/2014  14:13:10  PAGE 4


  C:017CH         LINE#         123
  C:0180H         LINE#         126
  C:0184H         LINE#         128
  C:0188H         LINE#         130
  C:018CH         LINE#         132
  C:0190H         LINE#         134
  C:0194H         LINE#         136
  C:0198H         LINE#         138
  C:019CH         LINE#         140
  C:01A0H         LINE#         142
  C:01A4H         LINE#         144
  C:01A8H         LINE#         146
  C:01ACH         LINE#         148
  C:01B0H         LINE#         150
  C:01B4H         LINE#         152
  -------         ENDMOD        USBJMPTBL

*** WARNING L1: UNRESOLVED EXTERNAL SYMBOL
    SYMBOL:  ISR_SUDAV
    MODULE:  .\USBJmpTb.OBJ (USBJMPTBL)

*** WARNING L1: UNRESOLVED EXTERNAL SYMBOL
    SYMBOL:  ISR_SOF
    MODULE:  .\USBJmpTb.OBJ (USBJMPTBL)

*** WARNING L1: UNRESOLVED EXTERNAL SYMBOL
    SYMBOL:  ISR_SUTOK
    MODULE:  .\USBJmpTb.OBJ (USBJMPTBL)

*** WARNING L1: UNRESOLVED EXTERNAL SYMBOL
    SYMBOL:  ISR_SUSP
    MODULE:  .\USBJmpTb.OBJ (USBJMPTBL)

*** WARNING L1: UNRESOLVED EXTERNAL SYMBOL
    SYMBOL:  ISR_URES
    MODULE:  .\USBJmpTb.OBJ (USBJMPTBL)

*** WARNING L1: UNRESOLVED EXTERNAL SYMBOL
    SYMBOL:  ISR_HIGHSPEED
    MODULE:  .\USBJmpTb.OBJ (USBJMPTBL)

*** WARNING L1: UNRESOLVED EXTERNAL SYMBOL
    SYMBOL:  ISR_EP0ACK
    MODULE:  .\USBJmpTb.OBJ (USBJMPTBL)

*** WARNING L1: UNRESOLVED EXTERNAL SYMBOL
    SYMBOL:  ISR_STUB
    MODULE:  .\USBJmpTb.OBJ (USBJMPTBL)

*** WARNING L1: UNRESOLVED EXTERNAL SYMBOL
    SYMBOL:  ISR_EP0IN
    MODULE:  .\USBJmpTb.OBJ (USBJMPTBL)

*** WARNING L1: UNRESOLVED EXTERNAL SYMBOL
    SYMBOL:  ISR_EP0OUT
    MODULE:  .\USBJmpTb.OBJ (USBJMPTBL)

BL51 BANKED LINKER/LOCATER V5.03                                                      06/13/2014  14:13:10  PAGE 5


*** WARNING L1: UNRESOLVED EXTERNAL SYMBOL
    SYMBOL:  ISR_EP1IN
    MODULE:  .\USBJmpTb.OBJ (USBJMPTBL)

*** WARNING L1: UNRESOLVED EXTERNAL SYMBOL
    SYMBOL:  ISR_EP1OUT
    MODULE:  .\USBJmpTb.OBJ (USBJMPTBL)

*** WARNING L1: UNRESOLVED EXTERNAL SYMBOL
    SYMBOL:  ISR_EP2INOUT
    MODULE:  .\USBJmpTb.OBJ (USBJMPTBL)

*** WARNING L1: UNRESOLVED EXTERNAL SYMBOL
    SYMBOL:  ISR_EP4INOUT
    MODULE:  .\USBJmpTb.OBJ (USBJMPTBL)

*** WARNING L1: UNRESOLVED EXTERNAL SYMBOL
    SYMBOL:  ISR_EP6INOUT
    MODULE:  .\USBJmpTb.OBJ (USBJMPTBL)

*** WARNING L1: UNRESOLVED EXTERNAL SYMBOL
    SYMBOL:  ISR_EP8INOUT
    MODULE:  .\USBJmpTb.OBJ (USBJMPTBL)

*** WARNING L1: UNRESOLVED EXTERNAL SYMBOL
    SYMBOL:  ISR_IBN
    MODULE:  .\USBJmpTb.OBJ (USBJMPTBL)

*** WARNING L1: UNRESOLVED EXTERNAL SYMBOL
    SYMBOL:  ISR_EP0PINGNAK
    MODULE:  .\USBJmpTb.OBJ (USBJMPTBL)

*** WARNING L1: UNRESOLVED EXTERNAL SYMBOL
    SYMBOL:  ISR_EP1PINGNAK
    MODULE:  .\USBJmpTb.OBJ (USBJMPTBL)

*** WARNING L1: UNRESOLVED EXTERNAL SYMBOL
    SYMBOL:  ISR_EP2PINGNAK
    MODULE:  .\USBJmpTb.OBJ (USBJMPTBL)

*** WARNING L1: UNRESOLVED EXTERNAL SYMBOL
    SYMBOL:  ISR_EP4PINGNAK
    MODULE:  .\USBJmpTb.OBJ (USBJMPTBL)

*** WARNING L1: UNRESOLVED EXTERNAL SYMBOL
    SYMBOL:  ISR_EP6PINGNAK
    MODULE:  .\USBJmpTb.OBJ (USBJMPTBL)

*** WARNING L1: UNRESOLVED EXTERNAL SYMBOL
    SYMBOL:  ISR_EP8PINGNAK
    MODULE:  .\USBJmpTb.OBJ (USBJMPTBL)

*** WARNING L1: UNRESOLVED EXTERNAL SYMBOL
    SYMBOL:  ISR_ERRORLIMIT
    MODULE:  .\USBJmpTb.OBJ (USBJMPTBL)

*** WARNING L1: UNRESOLVED EXTERNAL SYMBOL
BL51 BANKED LINKER/LOCATER V5.03                                                      06/13/2014  14:13:10  PAGE 6


    SYMBOL:  ISR_EP2PIDERROR
    MODULE:  .\USBJmpTb.OBJ (USBJMPTBL)

*** WARNING L1: UNRESOLVED EXTERNAL SYMBOL
    SYMBOL:  ISR_EP4PIDERROR
    MODULE:  .\USBJmpTb.OBJ (USBJMPTBL)

*** WARNING L1: UNRESOLVED EXTERNAL SYMBOL
    SYMBOL:  ISR_EP6PIDERROR
    MODULE:  .\USBJmpTb.OBJ (USBJMPTBL)

*** WARNING L1: UNRESOLVED EXTERNAL SYMBOL
    SYMBOL:  ISR_EP8PIDERROR
    MODULE:  .\USBJmpTb.OBJ (USBJMPTBL)

*** WARNING L1: UNRESOLVED EXTERNAL SYMBOL
    SYMBOL:  ISR_EP2PFLAG
    MODULE:  .\USBJmpTb.OBJ (USBJMPTBL)

*** WARNING L1: UNRESOLVED EXTERNAL SYMBOL
    SYMBOL:  ISR_EP4PFLAG
    MODULE:  .\USBJmpTb.OBJ (USBJMPTBL)

*** WARNING L1: UNRESOLVED EXTERNAL SYMBOL
    SYMBOL:  ISR_EP6PFLAG
    MODULE:  .\USBJmpTb.OBJ (USBJMPTBL)

*** WARNING L1: UNRESOLVED EXTERNAL SYMBOL
    SYMBOL:  ISR_EP8PFLAG
    MODULE:  .\USBJmpTb.OBJ (USBJMPTBL)

*** WARNING L1: UNRESOLVED EXTERNAL SYMBOL
    SYMBOL:  ISR_EP2EFLAG
    MODULE:  .\USBJmpTb.OBJ (USBJMPTBL)

*** WARNING L1: UNRESOLVED EXTERNAL SYMBOL
    SYMBOL:  ISR_EP4EFLAG
    MODULE:  .\USBJmpTb.OBJ (USBJMPTBL)

*** WARNING L1: UNRESOLVED EXTERNAL SYMBOL
    SYMBOL:  ISR_EP6EFLAG
    MODULE:  .\USBJmpTb.OBJ (USBJMPTBL)

*** WARNING L1: UNRESOLVED EXTERNAL SYMBOL
    SYMBOL:  ISR_EP8EFLAG
    MODULE:  .\USBJmpTb.OBJ (USBJMPTBL)

*** WARNING L1: UNRESOLVED EXTERNAL SYMBOL
    SYMBOL:  ISR_EP2FFLAG
    MODULE:  .\USBJmpTb.OBJ (USBJMPTBL)

*** WARNING L1: UNRESOLVED EXTERNAL SYMBOL
    SYMBOL:  ISR_EP4FFLAG
    MODULE:  .\USBJmpTb.OBJ (USBJMPTBL)

*** WARNING L1: UNRESOLVED EXTERNAL SYMBOL
    SYMBOL:  ISR_EP6FFLAG
BL51 BANKED LINKER/LOCATER V5.03                                                      06/13/2014  14:13:10  PAGE 7


    MODULE:  .\USBJmpTb.OBJ (USBJMPTBL)

*** WARNING L1: UNRESOLVED EXTERNAL SYMBOL
    SYMBOL:  ISR_EP8FFLAG
    MODULE:  .\USBJmpTb.OBJ (USBJMPTBL)

*** WARNING L1: UNRESOLVED EXTERNAL SYMBOL
    SYMBOL:  ISR_GPIFCOMPLETE
    MODULE:  .\USBJmpTb.OBJ (USBJMPTBL)

*** WARNING L1: UNRESOLVED EXTERNAL SYMBOL
    SYMBOL:  ISR_GPIFWAVEFORM
    MODULE:  .\USBJmpTb.OBJ (USBJMPTBL)

*** WARNING L2: REFERENCE MADE TO UNRESOLVED EXTERNAL
    SYMBOL:  ISR_SUDAV
    MODULE:  .\USBJmpTb.OBJ (USBJMPTBL)
    ADDRESS: 0101H

*** WARNING L2: REFERENCE MADE TO UNRESOLVED EXTERNAL
    SYMBOL:  ISR_SOF
    MODULE:  .\USBJmpTb.OBJ (USBJMPTBL)
    ADDRESS: 0105H

*** WARNING L2: REFERENCE MADE TO UNRESOLVED EXTERNAL
    SYMBOL:  ISR_SUTOK
    MODULE:  .\USBJmpTb.OBJ (USBJMPTBL)
    ADDRESS: 0109H

*** WARNING L2: REFERENCE MADE TO UNRESOLVED EXTERNAL
    SYMBOL:  ISR_SUSP
    MODULE:  .\USBJmpTb.OBJ (USBJMPTBL)
    ADDRESS: 010DH

*** WARNING L2: REFERENCE MADE TO UNRESOLVED EXTERNAL
    SYMBOL:  ISR_URES
    MODULE:  .\USBJmpTb.OBJ (USBJMPTBL)
    ADDRESS: 0111H

*** WARNING L2: REFERENCE MADE TO UNRESOLVED EXTERNAL
    SYMBOL:  ISR_HIGHSPEED
    MODULE:  .\USBJmpTb.OBJ (USBJMPTBL)
    ADDRESS: 0115H

*** WARNING L2: REFERENCE MADE TO UNRESOLVED EXTERNAL
    SYMBOL:  ISR_EP0ACK
    MODULE:  .\USBJmpTb.OBJ (USBJMPTBL)
    ADDRESS: 0119H

*** WARNING L2: REFERENCE MADE TO UNRESOLVED EXTERNAL
    SYMBOL:  ISR_STUB
    MODULE:  .\USBJmpTb.OBJ (USBJMPTBL)
    ADDRESS: 011DH

*** WARNING L2: REFERENCE MADE TO UNRESOLVED EXTERNAL
    SYMBOL:  ISR_EP0IN
    MODULE:  .\USBJmpTb.OBJ (USBJMPTBL)
BL51 BANKED LINKER/LOCATER V5.03                                                      06/13/2014  14:13:10  PAGE 8


    ADDRESS: 0121H

*** WARNING L2: REFERENCE MADE TO UNRESOLVED EXTERNAL
    SYMBOL:  ISR_EP0OUT
    MODULE:  .\USBJmpTb.OBJ (USBJMPTBL)
    ADDRESS: 0125H

*** WARNING L2: REFERENCE MADE TO UNRESOLVED EXTERNAL
    SYMBOL:  ISR_EP1IN
    MODULE:  .\USBJmpTb.OBJ (USBJMPTBL)
    ADDRESS: 0129H

*** WARNING L2: REFERENCE MADE TO UNRESOLVED EXTERNAL
    SYMBOL:  ISR_EP1OUT
    MODULE:  .\USBJmpTb.OBJ (USBJMPTBL)
    ADDRESS: 012DH

*** WARNING L2: REFERENCE MADE TO UNRESOLVED EXTERNAL
    SYMBOL:  ISR_EP2INOUT
    MODULE:  .\USBJmpTb.OBJ (USBJMPTBL)
    ADDRESS: 0131H

*** WARNING L2: REFERENCE MADE TO UNRESOLVED EXTERNAL
    SYMBOL:  ISR_EP4INOUT
    MODULE:  .\USBJmpTb.OBJ (USBJMPTBL)
    ADDRESS: 0135H

*** WARNING L2: REFERENCE MADE TO UNRESOLVED EXTERNAL
    SYMBOL:  ISR_EP6INOUT
    MODULE:  .\USBJmpTb.OBJ (USBJMPTBL)
    ADDRESS: 0139H

*** WARNING L2: REFERENCE MADE TO UNRESOLVED EXTERNAL
    SYMBOL:  ISR_EP8INOUT
    MODULE:  .\USBJmpTb.OBJ (USBJMPTBL)
    ADDRESS: 013DH

*** WARNING L2: REFERENCE MADE TO UNRESOLVED EXTERNAL
    SYMBOL:  ISR_IBN
    MODULE:  .\USBJmpTb.OBJ (USBJMPTBL)
    ADDRESS: 0141H

*** WARNING L2: REFERENCE MADE TO UNRESOLVED EXTERNAL
    SYMBOL:  ISR_STUB
    MODULE:  .\USBJmpTb.OBJ (USBJMPTBL)
    ADDRESS: 0145H

*** WARNING L2: REFERENCE MADE TO UNRESOLVED EXTERNAL
    SYMBOL:  ISR_EP0PINGNAK
    MODULE:  .\USBJmpTb.OBJ (USBJMPTBL)
    ADDRESS: 0149H

*** WARNING L2: REFERENCE MADE TO UNRESOLVED EXTERNAL
    SYMBOL:  ISR_EP1PINGNAK
    MODULE:  .\USBJmpTb.OBJ (USBJMPTBL)
    ADDRESS: 014DH

BL51 BANKED LINKER/LOCATER V5.03                                                      06/13/2014  14:13:10  PAGE 9


*** WARNING L2: REFERENCE MADE TO UNRESOLVED EXTERNAL
    SYMBOL:  ISR_EP2PINGNAK
    MODULE:  .\USBJmpTb.OBJ (USBJMPTBL)
    ADDRESS: 0151H

*** WARNING L2: REFERENCE MADE TO UNRESOLVED EXTERNAL
    SYMBOL:  ISR_EP4PINGNAK
    MODULE:  .\USBJmpTb.OBJ (USBJMPTBL)
    ADDRESS: 0155H

*** WARNING L2: REFERENCE MADE TO UNRESOLVED EXTERNAL
    SYMBOL:  ISR_EP6PINGNAK
    MODULE:  .\USBJmpTb.OBJ (USBJMPTBL)
    ADDRESS: 0159H

*** WARNING L2: REFERENCE MADE TO UNRESOLVED EXTERNAL
    SYMBOL:  ISR_EP8PINGNAK
    MODULE:  .\USBJmpTb.OBJ (USBJMPTBL)
    ADDRESS: 015DH

*** WARNING L2: REFERENCE MADE TO UNRESOLVED EXTERNAL
    SYMBOL:  ISR_ERRORLIMIT
    MODULE:  .\USBJmpTb.OBJ (USBJMPTBL)
    ADDRESS: 0161H

*** WARNING L2: REFERENCE MADE TO UNRESOLVED EXTERNAL
    SYMBOL:  ISR_STUB
    MODULE:  .\USBJmpTb.OBJ (USBJMPTBL)
    ADDRESS: 0165H

*** WARNING L2: REFERENCE MADE TO UNRESOLVED EXTERNAL
    SYMBOL:  ISR_STUB
    MODULE:  .\USBJmpTb.OBJ (USBJMPTBL)
    ADDRESS: 0169H

*** WARNING L2: REFERENCE MADE TO UNRESOLVED EXTERNAL
    SYMBOL:  ISR_STUB
    MODULE:  .\USBJmpTb.OBJ (USBJMPTBL)
    ADDRESS: 016DH

*** WARNING L2: REFERENCE MADE TO UNRESOLVED EXTERNAL
    SYMBOL:  ISR_EP2PIDERROR
    MODULE:  .\USBJmpTb.OBJ (USBJMPTBL)
    ADDRESS: 0171H

*** WARNING L2: REFERENCE MADE TO UNRESOLVED EXTERNAL
    SYMBOL:  ISR_EP4PIDERROR
    MODULE:  .\USBJmpTb.OBJ (USBJMPTBL)
    ADDRESS: 0175H

*** WARNING L2: REFERENCE MADE TO UNRESOLVED EXTERNAL
    SYMBOL:  ISR_EP6PIDERROR
    MODULE:  .\USBJmpTb.OBJ (USBJMPTBL)
    ADDRESS: 0179H

*** WARNING L2: REFERENCE MADE TO UNRESOLVED EXTERNAL
    SYMBOL:  ISR_EP8PIDERROR
BL51 BANKED LINKER/LOCATER V5.03                                                      06/13/2014  14:13:10  PAGE 10


    MODULE:  .\USBJmpTb.OBJ (USBJMPTBL)
    ADDRESS: 017DH

*** WARNING L2: REFERENCE MADE TO UNRESOLVED EXTERNAL
    SYMBOL:  ISR_EP2PFLAG
    MODULE:  .\USBJmpTb.OBJ (USBJMPTBL)
    ADDRESS: 0181H

*** WARNING L2: REFERENCE MADE TO UNRESOLVED EXTERNAL
    SYMBOL:  ISR_EP4PFLAG
    MODULE:  .\USBJmpTb.OBJ (USBJMPTBL)
    ADDRESS: 0185H

*** WARNING L2: REFERENCE MADE TO UNRESOLVED EXTERNAL
    SYMBOL:  ISR_EP6PFLAG
    MODULE:  .\USBJmpTb.OBJ (USBJMPTBL)
    ADDRESS: 0189H

*** WARNING L2: REFERENCE MADE TO UNRESOLVED EXTERNAL
    SYMBOL:  ISR_EP8PFLAG
    MODULE:  .\USBJmpTb.OBJ (USBJMPTBL)
    ADDRESS: 018DH

*** WARNING L2: REFERENCE MADE TO UNRESOLVED EXTERNAL
    SYMBOL:  ISR_EP2EFLAG
    MODULE:  .\USBJmpTb.OBJ (USBJMPTBL)
    ADDRESS: 0191H

*** WARNING L2: REFERENCE MADE TO UNRESOLVED EXTERNAL
    SYMBOL:  ISR_EP4EFLAG
    MODULE:  .\USBJmpTb.OBJ (USBJMPTBL)
    ADDRESS: 0195H

*** WARNING L2: REFERENCE MADE TO UNRESOLVED EXTERNAL
    SYMBOL:  ISR_EP6EFLAG
    MODULE:  .\USBJmpTb.OBJ (USBJMPTBL)
    ADDRESS: 0199H

*** WARNING L2: REFERENCE MADE TO UNRESOLVED EXTERNAL
    SYMBOL:  ISR_EP8EFLAG
    MODULE:  .\USBJmpTb.OBJ (USBJMPTBL)
    ADDRESS: 019DH

*** WARNING L2: REFERENCE MADE TO UNRESOLVED EXTERNAL
    SYMBOL:  ISR_EP2FFLAG
    MODULE:  .\USBJmpTb.OBJ (USBJMPTBL)
    ADDRESS: 01A1H

*** WARNING L2: REFERENCE MADE TO UNRESOLVED EXTERNAL
    SYMBOL:  ISR_EP4FFLAG
    MODULE:  .\USBJmpTb.OBJ (USBJMPTBL)
    ADDRESS: 01A5H

*** WARNING L2: REFERENCE MADE TO UNRESOLVED EXTERNAL
    SYMBOL:  ISR_EP6FFLAG
    MODULE:  .\USBJmpTb.OBJ (USBJMPTBL)
    ADDRESS: 01A9H
BL51 BANKED LINKER/LOCATER V5.03                                                      06/13/2014  14:13:10  PAGE 11



*** WARNING L2: REFERENCE MADE TO UNRESOLVED EXTERNAL
    SYMBOL:  ISR_EP8FFLAG
    MODULE:  .\USBJmpTb.OBJ (USBJMPTBL)
    ADDRESS: 01ADH

*** WARNING L2: REFERENCE MADE TO UNRESOLVED EXTERNAL
    SYMBOL:  ISR_GPIFCOMPLETE
    MODULE:  .\USBJmpTb.OBJ (USBJMPTBL)
    ADDRESS: 01B1H

*** WARNING L2: REFERENCE MADE TO UNRESOLVED EXTERNAL
    SYMBOL:  ISR_GPIFWAVEFORM
    MODULE:  .\USBJmpTb.OBJ (USBJMPTBL)
    ADDRESS: 01B5H

******************************************************************************
* RESTRICTED VERSION WITH 1000H BYTE CODE SIZE LIMIT; USED: 0101H BYTE ( 6%) *
******************************************************************************

Program Size: data=9.0 xdata=0 code=249
LINK/LOCATE RUN COMPLETE.  88 WARNING(S),  0 ERROR(S)
